:100000000C945B000C9483000C9483000C9483008C
:100010000C9483000C9483000C9483000C94830054
:100020000C9483000C9483000C9483000C94830044
:100030000C9483000C9483000C9483000C94830034
:100040000C94A90A0C9483000C94FB0C0C94830070
:100050000C9483000C9483000C9483000C94830014
:100060000C9483000C948300000024272A000025B0
:10007000282B000023262904040404040404040299
:100080000202020202030303030303010204081035
:100090002040800102040810200102040810200002
:1000A0000000070002010000030406000000000039
:1000B00000000000A80A11241FBECFEFD4E0DEBF6D
:1000C000CDBF11E0A0E0B1E0EEEFFCE102C0059091
:1000D0000D92AC34B107D9F712E0ACE4B1E001C045
:1000E0001D92AC30B107E1F710E0C6EBD0E004C0E0
:1000F0002297FE010E947A0EC43BD107C9F70E94E5
:100100004B090C947E0E0C94000010925901109231
:100110005801E0E0F0E0EE0FFF1FE45FFE4F61E00A
:1001200080810E94360CE0915801F091590131967E
:10013000F0935901E0935801E430F10564F3089518
:100140001F93CF93DF93182FC7E0D0E060E080913A
:1001500004010E94360C212F332781E090E00C2E01
:1001600002C0880F991F0A94E2F782239323892BF8
:1001700011F061E001C060E0809100010E94360C46
:1001800061E0809104010E94360C21978FEFCF3FF0
:10019000D807E1F6DF91CF911F910895DF92EF929A
:1001A000FF920F931F93CF93DF93F82EE62ED42E5A
:1001B00060E0809102010E94360CC0910A01D0914A
:1001C0000B0107C080E00E94A00080E00E94A00018
:1001D00021970F2D11270C171D07A4F38E2D0E94B8
:1001E000A0008D2D0E94A000E80106C080E00E94C2
:1001F000A00080E00E94A00021971C161D06B4F309
:1002000060E0809102010E94360C61E08091020161
:100210000E94360CDF91CF911F910F91FF90EF90CC
:10022000DF9008950F931F93CF93DF93082F162F1E
:1002300060E0809102010E94360CC1E0D0E007C06E
:10024000802F0E94A000812F0E94A0002196809103
:100250000A0190910B018C179D0794F760E0809143
:1002600002010E94360C61E0809102010E94360C6E
:10027000DF91CF911F910F9108950F931F93182F26
:10028000062F60E0809102010E94360C812F0E94AF
:10029000A000802F0E94A00060E0809102010E94D7
:1002A000360C61E0809102010E94360C1F910F9183
:1002B00008956FEF82E00E943D016FEF83E00E949E
:1002C0003D016FEF81E00E943D016FEF84E00E94ED
:1002D0003D016FEF88E00E943D016FEF85E00E94D5
:1002E0003D016FEF87E00E943D016FEF86E00E94C5
:1002F0003D01089561E0809100010E94CC0B61E016
:10030000809104010E94CC0B61E0809102010E9467
:10031000CC0B60E875E280E090E00E94810C61E027
:100320008DE00E94360C67E080911E010E94120150
:1003300060E080911C010E94120161E080911F0128
:100340000E94120160E0809120010E94120181E070
:1003500090E090934D0180934C0160E00E94120167
:1003600080914C0190914D01019690934D018093A5
:100370004C01893091058CF36FE080911D010E9442
:1003800012016091210182E00E943D0160912101F2
:1003900088E00E943D016091370181E00E943D01AB
:1003A0006091370187E00E943D016091370184E050
:1003B0000E943D016091370186E00E943D016091FD
:1003C000210183E00E943D016091210185E00E94AE
:1003D0003D010895CF93DF9320916C0130916D0121
:1003E00080916E0190916F010196821793070CF036
:1003F0007EC0283031050CF47AC010927B01109237
:100400007A0110925D0110925C0110925F011092CE
:100410005E011092510110925001109253011092FE
:1004200052011092610110926001109263011092CA
:10043000620110926D0110926C0110926F01109286
:100440006E01809154019091550101969093550150
:10045000809354016091370184E00E943D01E09156
:100460005201F0915301EE0FFF1FE95CFE4F6081D6
:1004700081E00E943D01E0915C01F0915D01EE0F91
:10048000FF1FEF5DFE4F608185E00E943D01E0911E
:100490006001F0916101EE0FFF1FEF5DFE4F608183
:1004A00083E00E943D01E0915E01F0915F01EE0F5B
:1004B000FF1FEF5DFE4F608188E00E943D01E091EB
:1004C0006201F0916301EE0FFF1FEF5DFE4F60814F
:1004D00082E00E943D01E0915401F0915501EE0F40
:1004E000FF1FE95CFE4F608186E00E943D01209184
:1004F0006E0130916F0180916C0190916D010196B8
:10050000821793070CF07EC0283031050CF47AC0B6
:1005100010927B0110927A0110925D0110925C01A1
:1005200010925F0110925E011092510110925001E1
:1005300010925301109252011092610110926001C9
:10054000109263011092620110926D0110926C0181
:1005500010926F0110926E01809156019091570197
:10056000019690935701809356016091370184E082
:100570000E943D01E0915201F0915301EE0FFF1FE7
:10058000E95CFE4F608181E00E943D01E0915C01E9
:10059000F0915D01EE0FFF1FEF5DFE4F608185E082
:1005A0000E943D01E0916001F0916101EE0FFF1F9B
:1005B000EF5DFE4F608183E00E943D01E0915E01AE
:1005C000F0915F01EE0FFF1FEF5DFE4F608188E04D
:1005D0000E943D01E0916201F0916301EE0FFF1F67
:1005E000EF5DFE4F608182E00E943D01E091560187
:1005F000F0915701EE0FFF1FE95CFE4F608187E02D
:100600000E943D018091500190915101069709F09F
:10061000BAC08091520190915301069709F0B3C07E
:1006200080917E0190917F01892B09F0ACC0C1E0DF
:10063000D0E0D0937B01C0937A01809106010E94A3
:100640005A0B803891050CF04AC08091740190914A
:100650007501892B09F043C0D0937501C0937401D3
:1006600080915C0190915D01019690935D01809372
:100670005C010A979CF010925D0110925C018091E0
:1006800060019091610101969093610180936001F6
:100690000A9724F0109261011092600180916C0120
:1006A00090916D01019690936D0180936C01E091A2
:1006B0006001F0916101EE0FFF1FEF5DFE4F608161
:1006C00083E00E943D01E0915C01F0915D01EE0F3D
:1006D000FF1FEF5DFE4F608185E00E943D0180912C
:1006E00008010E945A0B803891050CF04CC0809193
:1006F000760190917701892B09F045C081E090E067
:10070000909377018093760180915E0190915F01D3
:10071000019690935F0180935E010A979CF010927E
:100720005F0110925E0180916201909163010196D8
:1007300090936301809362010A9724F01092630101
:100740001092620180916E0190916F0101969093D9
:100750006F0180936E01E0916201F0916301EE0FF1
:10076000FF1FEF5DFE4F608182E00E943D01E0913E
:100770005E01F0915F01EE0FFF1FEF5DFE4F6081A4
:1007800088E00E943D01DF91CF910895CF93DF93E0
:10079000809108010E945A0B803891050CF0CCC260
:1007A000809106010E945A0B803891050CF0C4C25A
:1007B0008091780190917901892B09F0BDC281E087
:1007C00090E090937901809378010E94CE0A709313
:1007D0007D0160937C0131C0809106010E945A0B1B
:1007E000803891050CF0B0C2809178019091790128
:1007F000019709F0A9C20E94CE0A20917C01309194
:100800007D01621B730B709381016093800183E80B
:1008100091E00E947E0A11C0809106010E945A0B4D
:100820008D5F934054F08091780190917901019708
:1008300021F41092790110927801809180019091B9
:100840008101815D97400CF486C06091210182E0B6
:100850000E943D016091210188E00E943D0160916C
:10086000370181E00E943D016091370187E00E94DD
:100870003D016091370184E00E943D0160913701A4
:1008800086E00E943D016091210183E00E943D01CC
:100890006091210185E00E943D0180917E0190914F
:1008A0007F01892B39F481E090E090937F01809360
:1008B0007E0104C010927F0110927E0110927D0192
:1008C00010927C0110925D0110925C0110925F0108
:1008D00010925E011092610110926001109263010A
:1008E00010926201109265011092640110926701EA
:1008F00010926601109269011092680110926B01CA
:1009000010926A0110926D0110926C0110926F01A9
:1009100010926E0110927101109270011092730189
:100920001092720110927B0110927A011092810153
:1009300010928001109257011092560110925501A9
:1009400010925401109253011092520110925101D1
:10095000109250013EC1209170013091710180913F
:100960007201909173010196821793070CF092C067
:100970002C3031050CF48EC0109265011092640188
:10098000109267011092660110926901109268013D
:1009900010926B0110926A01109271011092700115
:1009A000109273011092720180915401909155013F
:1009B000019690935501809354010297B9F41092D7
:1009C00055011092540110925701109256018091D6
:1009D00050019091510101969093510180935001E3
:1009E0000A9721F41092510110925001E0915401A4
:1009F000F0915501EE0FFF1FE95CFE4F608184E02E
:100A00000E943D01E0915601F0915701EE0FFF1F4A
:100A1000E95CFE4F608181E00E943D01E09164014C
:100A2000F0916501EE0FFF1FEF5DFE4F608185E0E5
:100A30000E943D01E0916801F0916901EE0FFF1FF6
:100A4000EF5DFE4F608183E00E943D01E091660111
:100A5000F0916701EE0FFF1FEF5DFE4F608188E0B0
:100A60000E943D01E0916A01F0916B01EE0FFF1FC2
:100A7000EF5DFE4F608182E00E943D01E0915001F8
:100A8000F0915101EE0FFF1FE95CFE4F608186E09F
:100A90000E943D012091720130917301809170019B
:100AA000909171010196821793070CF092C02C303F
:100AB00031050CF48EC01092650110926401109201
:100AC00067011092660110926901109268011092FC
:100AD0006B0110926A0110927101109270011092D4
:100AE0007301109272018091560190915701019605
:100AF00090935701809356010297B9F410925501D3
:100B00001092540110925701109256018091520197
:100B100090915301019690935301809352010A974B
:100B200021F41092530110925201E0915401F0917E
:100B30005501EE0FFF1FE95CFE4F608184E00E94CB
:100B40003D01E0915601F0915701EE0FFF1FE95C66
:100B5000FE4F608181E00E943D01E0916401F091CF
:100B60006501EE0FFF1FEF5DFE4F608185E00E9483
:100B70003D01E0916801F0916901EE0FFF1FEF5D0B
:100B8000FE4F608183E00E943D01E0916601F0919B
:100B90006701EE0FFF1FEF5DFE4F608188E00E944E
:100BA0003D01E0916A01F0916B01EE0FFF1FEF5DD7
:100BB000FE4F608182E00E943D01E0915201F09180
:100BC0005301EE0FFF1FE95CFE4F608187E00E943A
:100BD0003D01C0917E01D0917F01C130D10509F066
:100BE000BCC0D0937B01C0937A01809106010E9422
:100BF0005A0B803891050CF04AC080917401909195
:100C00007501892B09F043C0D0937501C09374011D
:100C100080916401909165010196909365018093A4
:100C200064010A979CF01092650110926401809112
:100C30006801909169010196909369018093680120
:100C40000A9724F010926901109268018091700156
:100C50009091710101969093710180937001E091E0
:100C60006801F0916901EE0FFF1FEF5DFE4F60819B
:100C700083E00E943D01E0916401F0916501EE0F77
:100C8000FF1FEF5DFE4F608185E00E943D01809176
:100C900008010E945A0B803891050CF05EC08091CB
:100CA000760190917701892B09F057C081E090E09F
:100CB000909377018093760180916601909167010E
:100CC000019690936701809366010A979CF01092B9
:100CD00067011092660180916A0190916B01019603
:100CE00090936B0180936A010A9724F010926B0134
:100CF00010926A0180917201909173010196909314
:100D0000730180937201E0916A01F0916B01EE0F23
:100D1000FF1FEF5DFE4F608182E00E943D01E09188
:100D20006601F0916701EE0FFF1FEF5DFE4F6081DE
:100D300088E00E943D0111C0809108010E945A0B79
:100D4000803891050CF448CD809108010E945A0B1F
:100D50008D5F93400CF067CD5FCDDF91CF9108950B
:100D6000809108010E945A0B803891050CF070C1E7
:100D70008091760190917701892B09F069C180916A
:100D80007A0190917B01892B09F062C180917E01EB
:100D900090917F01892B09F05BC181E090E09093F5
:100DA00077018093760180915E0190915F010097B9
:100DB00071F48FE090E090935F0180935E01609109
:100DC000230182E00E943D0160912B0132C18F30EE
:100DD000910549F48EE190E090935F0180935E016C
:100DE0006091270121C18E31910539F488E290E0AC
:100DF00090935F0180935E012EC08832910509F0C7
:100E0000A2C020915C0130915D012832310571F45E
:100E100089E290E090935F0180935E0160912901E7
:100E200082E00E943D016091350103C12932310504
:100E3000A9F490935D0180935C0190935F0180938E
:100E40005E016091290183E00E943D0160912101D2
:100E500085E00E943D0160912901E6C010925F018A
:100E600010925E0110925D0110925C01809152011E
:100E7000909153018930910529F4109253011092F9
:100E8000520105C0019690935301809352016091E5
:100E9000210182E00E943D016091210188E00E94D1
:100EA0003D01E0915201F0915301E630F10539F432
:100EB0008091500190915101049724F033C0E730A4
:100EC000F10581F5109253011092520110925101D7
:100ED0001092500180915601909157010196909384
:100EE0005701809356016091370181E00E943D01D6
:100EF0006091370184E00E943D01E0915601F0913C
:100F00005701EA30F10539F4109257011092560159
:100F10006091370105C0EE0FFF1FE95CFE4F608155
:100F200087E006C0EE0FFF1FE95CFE4F608181E0A5
:100F30000E943D016091210183E00E943D0160918A
:100F4000210185E077C0899709F089C010925F017F
:100F500010925E0110925D0110925C01809152012D
:100F6000909153018930910529F410925301109208
:100F7000520105C0019690935301809352016091F4
:100F8000210183E00E943D016091210185E00E94E2
:100F90003D01E0915201F0915301E630F10539F441
:100FA0008091500190915101049724F033C0E730B3
:100FB000F10581F5109253011092520110925101E6
:100FC0001092500180915601909157010196909393
:100FD0005701809356016091370181E00E943D01E5
:100FE0006091370184E00E943D01E0915601F0914B
:100FF0005701EA30F10539F4109257011092560169
:101000006091370105C0EE0FFF1FE95CFE4F608164
:1010100087E006C0EE0FFF1FE95CFE4F608181E0B4
:101020000E943D016091210182E00E943D0160919A
:10103000210188E00E943D0108956AE070E080E0AF
:1010400090E00E94E60A10927701109276010895CE
:10105000809108010E945A0B8D5F934074F70895A8
:10106000809106010E945A0B803891050CF002C154
:101070008091740190917501892B09F0FBC08091DA
:101080007A0190917B01892B09F0F4C080917E0157
:1010900090917F01892B09F0EDC081E090E0909361
:1010A00075018093740180915C0190915D010097BE
:1010B00071F48FE090E090935D0180935C0160910A
:1010C000230183E00E943D0160912B011CC08F3001
:1010D000910549F48EE190E090935D0180935C016D
:1010E000609127010BC08E31910579F488E290E080
:1010F00090935D0180935C016091290183E00E94DF
:101100003D016091210185E0A7C08832910569F514
:1011100020915E0130915F012832310571F489E23E
:1011200090E090935D0180935C016091290183E0E0
:101130000E943D0160913501E6CF29323105C1F4AD
:1011400090935D0180935C0190935F0180935E01B9
:101150006091290183E00E943D016091210185E0B9
:101160000E943D016091290171C0899709F089C0F1
:1011700010925D0110925C0110925F0110925E016D
:1011800080915001909151018930910529F410927C
:1011900051011092500105C0019690935101809326
:1011A00050016091210183E00E943D016091210185
:1011B00085E00E943D01E0915001F0915101E6303F
:1011C000F10539F48091520190915301049724F074
:1011D00033C0E730F10581F51092530110925201AE
:1011E000109251011092500180915401909155013B
:1011F000019690935501809354016091370184E0EA
:101200000E943D016091370181E00E943D01E09123
:101210005401F0915501EA30F10539F4109255016D
:10122000109254016091370105C0EE0FFF1FE95C79
:10123000FE4F608186E006C0EE0FFF1FE95CFE4FA7
:10124000608184E00E943D016091210182E00E9462
:101250003D016091210188E00E943D0108956AE00E
:1012600070E080E090E00E94E60A10927501109212
:1012700074010895809106010E945A0B8D5F93407E
:1012800074F708950E94C6030E94EA010E94300884
:101290000E94B00608950E94150B0E947A010E94D8
:1012A0004209FDCF68EE73E080E090E00E94E60A1C
:1012B000809150019091510101969093510180933A
:1012C00050010A970CF443C0809152019091530150
:1012D000019690935301809352010A9724F0109243
:1012E000530110925201E0915201F0915301EE0F1F
:1012F000FF1FEF5DFE4F608182E00E943D01E091A3
:101300005201F0915301EE0FFF1FEF5DFE4F608120
:1013100083E00E943D01E0915201F0915301EE0FF4
:10132000FF1FE95CFE4F608181E00E943D01E0917A
:101330005201F0915301EE0FFF1FE95CFE4F6081F7
:1013400084E00E943D011092510110925001E09101
:101350005001F0915101EE0FFF1FEF5DFE4F6081D4
:1013600088E00E943D01E0915001F0915101EE0FA3
:10137000FF1FEF5DFE4F608185E00E943D01E0911F
:101380005001F0915101EE0FFF1FE95CFE4F6081AB
:1013900087E00E943D01E0915001F0915101EE0F74
:1013A000FF1FE95CFE4F608186E00E943D010895C9
:1013B00008950895CB01BA013327442755270E9489
:1013C000410D08952AE00E94DA090895AB016627CD
:1013D00077270E94E2090895862F0E94390D08950B
:1013E000862F0E94390D08950F931F938C016DE095
:1013F0000E94F0096AE0C8010E94F0091F910F9154
:1014000008950F931F938C010E94E209C8010E9466
:10141000F4091F910F9108950F931F938C010E945F
:10142000E609C8010E94F4091F910F9108950F93D6
:101430001F938C010E94EC09C8010E94F4091F91BE
:101440000F9108950F931F938C010E94F009C8011A
:101450000E94F4091F910F910895EF92FF920F934C
:101460001F93CF93DF93EC017A018B0177FF0BC0C1
:101470006DE20E94F00910950095F094E094E11C53
:10148000F11C011D111D2AE0B801A701CE010E9427
:10149000DA09DF91CF911F910F91FF90EF9008959E
:1014A0000F931F938C010E942D0AC8010E94F4091A
:1014B0001F910F9108952115310521F4642F0E9489
:1014C000F00908952A30310519F40E942D0A089573
:1014D0000E94DA0908950F931F938C010E945B0A02
:1014E000C8010E94F4091F910F910895AB0166276E
:1014F00057FD6095762F0E942D0A08950F931F9334
:101500008C010E94760AC8010E94F4091F910F9174
:101510000895CB010E94070E08950F931F938C012D
:101520000E94890AC8010E94F4091F910F91089531
:101530000E94F20C08950E94D30C08950E94C20CE0
:1015400099270895CB01BA010E94810C089508954E
:1015500008951F920F920FB60F9211248F939F93AD
:10156000AF93BF938091880190918901A0918A01E6
:10157000B0918B010196A11DB11D809388019093BC
:101580008901A0938A01B0938B01BF91AF919F9184
:101590008F910F900FBE0F901F901895609188014A
:1015A0007091890180918A0190918B0127E0660FEB
:1015B000771F881F991F2A95D1F72DE730E040E06B
:1015C00050E00E94270ECA01B9010895AF92BF9260
:1015D000CF92DF92EF92FF920F931F935B016C010A
:1015E0000E94CE0A7B018C010E94CE0A6E197F09EF
:1015F000800B910B6A157B058C059D05A8F31F9147
:101600000F91FF90EF90DF90CF90BF90AF90089533
:10161000019751F0880F991F880F991F02972FB7D4
:10162000F8940197F1F72FBF0895789410928801EC
:101630001092890110928A0110928B0184B5826008
:1016400084BD84B5816084BD85B5826085BD85B566
:10165000816085BDEEE6F0E0808181608083E1E815
:10166000F0E0808182608083808181608083E0E817
:10167000F0E0808181608083E1EBF0E08081846034
:101680008083E0EBF0E0808181608083EAE7F0E036
:10169000808184608083808182608083808181609A
:1016A00080838081806880831092C1000895809338
:1016B0004B01089590914B019295990F990F907C51
:1016C0008F70982B90937C0080917A008064809337
:1016D0007A0080917A0086FDFCCF2091780080917D
:1016E00079009927982F88273327822B932B0895E9
:1016F0001F93CF93DF93182FEB0161E00E94CC0B77
:10170000E12FFF27E156FF4F8491833051F4809100
:101710008000806880938000D0938900C093880007
:1017200037C0843051F480918000806280938000C3
:10173000D0938B00C0938A002BC0813029F484B5EC
:10174000806884BDC7BD24C0823029F484B580621E
:1017500084BDC8BD1DC0863041F48091B000806852
:101760008093B000C093B30013C0873041F48091E0
:10177000B00080628093B000C093B40009C0C0384C
:10178000D10514F460E001C061E0812F0E94360CA5
:10179000DF91CF911F910895282F3327C9018557D5
:1017A0009F4FFC01949129583F4FF9018491882360
:1017B00081F0E82FFF27E859FF4FE491FF276623C8
:1017C00029F4808190958923808308958081892BD5
:1017D00080830895482F5527CA0181569F4FFC01E9
:1017E0002491CA0185579F4FFC01949149585F4F3E
:1017F000FA013491332319F480E090E00895222314
:1018000031F1233021F4809180008F7705C024309E
:1018100031F4809180008F7D8093800018C021304A
:1018200019F484B58F7704C0223021F484B58F7DFC
:1018300084BD0DC0263021F48091B0008F7705C0A3
:10184000273029F48091B0008F7D8093B000E32F82
:10185000FF27EE58FF4FE491FF27808120E030E022
:10186000892311F021E030E0C9010895482F552760
:10187000CA0181569F4FFC012491CA0185579F4F91
:10188000FC01949149585F4FFA0134913323C1F11F
:10189000222331F1233021F4809180008F7705C01D
:1018A000243031F4809180008F7D8093800018C0B7
:1018B000213019F484B58F7704C0223021F484B527
:1018C0008F7D84BD0DC0263021F48091B0008F77CC
:1018D00005C0273029F48091B0008F7D8093B0003F
:1018E000E32FFF27E359FF4FE491FF27662329F4F5
:1018F000808190958923808308958081892B8083BE
:101900000895EF92FF920F931F937B018C0122E0C9
:1019100030E040E050E00E94490E205C3D4B404FDB
:101920005F4FCA01B901A80197010E94490E2150D9
:10193000304040405040BB2757FDBA95A52F942F0B
:10194000832F2F5F3F4F4F4F5F4F8093C500215034
:101950002093C400E1ECF0E080818061808380818D
:10196000886080838081806880831F910F91FF90C1
:10197000EF900895982F8091C00085FFFCCF909341
:10198000C60008958091840190918501209186017F
:1019900030918701821B930B80589F4F60E870E065
:1019A0000E94140E08954091860150918701809104
:1019B0008401909185018417950719F48FEF9FEFAB
:1019C0000895FA01E457FE4F2081CA01019660E8AC
:1019D00070E00E94140E9093870180938601822FFD
:1019E00099270895809186019091870190938501B0
:1019F0008093840108951F920F920FB60F921124C5
:101A00002F933F934F935F936F937F938F939F9306
:101A1000AF93BF93EF93FF934091C600E091840191
:101A2000F0918501CF01019660E870E00E94140EEC
:101A30009C0180918601909187012817390739F020
:101A4000E457FE4F40833093850120938401FF913A
:101A5000EF91BF91AF919F918F917F916F915F9126
:101A60004F913F912F910F900FBE0F901F9018959F
:101A70000895982F8091C00085FFFCCF9093C600F9
:101A800008952F923F924F925F926F927F928F9222
:101A90009F92AF92BF92CF92DF92EF92FF920F93FD
:101AA0001F93CF93DF93CDB7DEB7A0970FB6F8940F
:101AB000DEBF0FBECDBF6B017C0129013A0161156C
:101AC00071058105910541F48091C00085FFFCCF2F
:101AD00080E38093C60041C08824992454011E01EC
:101AE0000894211C311C8101080D191DC701B60184
:101AF000A30192010E94270EF80160830894811CC3
:101B0000911CA11CB11CC701B601A30192010E9446
:101B1000270E69017A01211531054105510519F793
:101B20009E012F5F3F4F14C0089481089108A108BF
:101B3000B108F901E80DF91DE081EA3010F4E05D2B
:101B400001C0E95C8091C00085FFFCCFE093C60036
:101B500081149104A104B10439F7A0960FB6F8944A
:101B6000DEBF0FBECDBFDF91CF911F910F91FF90D0
:101B7000EF90DF90CF90BF90AF909F908F907F902D
:101B80006F905F904F903F902F90089520E130E04C
:101B900040E050E00E94410D089528E030E040E030
:101BA00050E00E94410D089522E030E040E050E016
:101BB0000E94410D08958091C00085FFFCCF8AE00E
:101BC0008093C6000895EF92FF920F931F937B01BD
:101BD0008C0197FF0FC08091C00085FFFCCF8DE284
:101BE0008093C60010950095F094E094E11CF11CE0
:101BF000011D111D2AE030E040E050E0C801B701AE
:101C00000E94410D1F910F91FF90EF900895FC01EC
:101C100007C08091C00085FFFCCF31969093C6002D
:101C200090819923B1F7089597FB092E07260AD0D2
:101C300077FD04D049D006D000201AF47095619544
:101C40007F4F0895F6F7909581959F4F0895A1E2F3
:101C50001A2EAA1BBB1BFD010DC0AA1FBB1FEE1F26
:101C6000FF1FA217B307E407F50720F0A21BB30B71
:101C7000E40BF50B661F771F881F991F1A9469F7ED
:101C800060957095809590959B01AC01BD01CF0149
:101C9000089597FB092E05260ED057FD04D0D7DFF7
:101CA0000AD0001C38F450954095309521953F4F4F
:101CB0004F4F5F4F0895F6F7909580957095619519
:101CC0007F4F8F4F9F4F0895AA1BBB1B51E107C049
:101CD000AA1FBB1FA617B70710F0A61BB70B881FBC
:101CE000991F5A95A9F780959095BC01CD0108954B
:0E1CF000EE0FFF1F0590F491E02D0994FFCF39
:101CFE0002000300040003000200010001000200C4
:101D0E00030004000102030405060801090A0B0C76
:101D1E000FED0005007C005D009500D900F9000D67
:101D2E0000FD00DD00EF007E0030006D0079003315
:0C1D3E00005B005F0070007F007B000174
:00000001FF
